:020000040000FA
:020000001728BF
:08000800C000030EC1000B1B38
:100010000C1C0D285B200C1012288B1A0B1D1228AB
:1000200065200B11410E8300C00E400E090083169F
:10003000FF2390008312203084008001840A041F73
:100040001D28841E1D288316810196018C019F01A5
:100050009901831207309900900183168501851656
:10006000950195168B018B170B178C010C148312BD
:100070008510851A39284320432043204F204F20E4
:10008000432043203928FD30A1008F001B30A200FF
:100090008E001014FF30A00010184C280800FA3011
:1000A000A1008F00C930A2008E001014FF30A00004
:1000B000101858280800101021088F0022088E0000
:0C00C00002308506A00B10140800080098
:02400E00843FED
:0442000003000400B3
:00000001FF
